******************************************************************************
               TMS320C6x Linker PC v7.4.2                      
******************************************************************************
>> Linked Wed Jan 08 11:34:50 2014

OUTPUT FILE NAME:   <EMIF.out>
ENTRY POINT SYMBOL: "_c_int00"  address: 0c08fd20


MEMORY CONFIGURATION

         name            origin    length      used     unused   attr    fill
----------------------  --------  ---------  --------  --------  ----  --------
  VECTORS               00800000   00000200  00000000  00000200  RWIX
  LL2_RW_DATA           00800200   0003fe00  000043e4  0003ba1c  RWIX
  SL2                   0c000000   00100000  00090300  0006fd00  RWIX
  EMIF16_DATA           70000000   10000000  00000000  10000000  RWIX
  DDR3_CODE             80000000   01000000  00000000  01000000  RWIX
  DDR3_R_DATA           81000000   01000000  00000000  01000000  RWIX
  DDR3_RW_DATA          82000000   06000000  00000000  06000000  RWIX


SEGMENT ALLOCATION MAP

run origin  load origin   length   init length attrs members
----------  ----------- ---------- ----------- ----- -------
00800200    00800200    00002100   00002100    r--
  00800200    00800200    00002100   00002100    r-- .const
00802300    00802300    00001800   00000000    rw-
  00802300    00802300    00001000   00000000    rw- .stack
  00803300    00803300    00000800   00000000    rw- .sysmem
00803b00    00803b00    00000474   00000474    rw-
  00803b00    00803b00    00000474   00000474    rw- .fardata
00803f78    00803f78    00000338   00000218    rw-
  00803f78    00803f78    00000218   00000218    rw- .far
  00804190    00804190    00000120   00000000    rw- .cio
008042b0    008042b0    000000a8   0000009c    rw-
  008042b0    008042b0    0000009c   0000009c    rw- .neardata
  0080434c    0080434c    0000000c   00000000    rw- .bss
00804358    00804358    00000290   00000290    r--
  00804358    00804358    00000290   00000290    r-- .cinit
0c000000    0c000000    00080000   00000000    rw-
  0c000000    0c000000    00080000   00000000    rw- .far:testBuf
0c080000    0c080000    00010300   00010300    r-x
  0c080000    0c080000    00010300   00010300    r-x .text


SECTION ALLOCATION MAP

 output                                  attributes/
section   page    origin      length       input sections
--------  ----  ----------  ----------   ----------------
.const     0    00800200    00002100     
                  00800200    00001a34     KeyStone_common.obj (.const:.string)
                  00801c34    000001e8     EMIF_FLASH_mem_test.obj (.const:.string)
                  00801e1c    000001d1     flash_nand.obj (.const:.string)
                  00801fed    00000107     KeyStone_EMIF16_Init.obj (.const:.string)
                  008020f4    00000002     rts6600e_elf.lib : fputs.obj (.const:.string)
                  008020f6    00000002     --HOLE-- [fill = 0]
                  008020f8    00000101                      : ctype.obj (.const:.string:_ctypes_)
                  008021f9    0000007b     EMIF_NAND_FLASH_test.obj (.const:.string)
                  00802274    00000004     --HOLE-- [fill = 0]
                  00802278    00000038     KeyStone_common.obj (.const:$P$T0$1)
                  008022b0    0000002d     EMIF_main.obj (.const:.string)
                  008022dd    00000023     rts6600e_elf.lib : _printfi.obj (.const:.string)

.stack     0    00802300    00001000     UNINITIALIZED
                  00802300    00000008     rts6600e_elf.lib : boot.obj (.stack)
                  00802308    00000ff8     --HOLE--

.sysmem    0    00803300    00000800     UNINITIALIZED
                  00803300    00000008     rts6600e_elf.lib : memory.obj (.sysmem)
                  00803308    000007f8     --HOLE--

.fardata   0    00803b00    00000474     
                  00803b00    000001e0     rts6600e_elf.lib : defs.obj (.fardata:_ftable)
                  00803ce0    000000a0                      : lowlev.obj (.fardata:_stream)
                  00803d80    00000078                      : lowlev.obj (.fardata:_device)
                  00803df8    00000040     KeyStone_common.obj (.fardata:gstruMpuAddrRange)
                  00803e38    00000028     EMIF_NAND_FLASH_test.obj (.fardata)
                  00803e60    00000024     KeyStone_common.obj (.fardata:gpTimerRegs)
                  00803e84    00000004     rts6600e_elf.lib : defs.obj (.fardata)
                  00803e88    00000024     KeyStone_common.obj (.fardata:internal_exception_str)
                  00803eac    00000004     --HOLE--
                  00803eb0    00000020     KeyStone_common.obj (.fardata:bus_err_stat_str)
                  00803ed0    00000020     KeyStone_common.obj (.fardata:gCIC_EXC_EN_MASK)
                  00803ef0    00000020     KeyStone_common.obj (.fardata:gpMPU_regs)
                  00803f10    00000018     KeyStone_common.obj (.fardata:Peri_MPU_err_type_str)
                  00803f28    00000010     KeyStone_common.obj (.fardata:gpEDMA_TC_regs)
                  00803f38    0000000c     rts6600e_elf.lib : exit.obj (.fardata)
                  00803f44    0000000c                      : memory.obj (.fardata)
                  00803f50    0000000c     EMIF_FLASH_mem_test.obj (.fardata:uiDataPatternTable)
                  00803f5c    00000004     --HOLE--
                  00803f60    00000008     KeyStone_common.obj (.fardata:Ns_str)
                  00803f68    00000008     rts6600e_elf.lib : _lock.obj (.fardata)
                  00803f70    00000004     KeyStone_common.obj (.fardata:gpEDMA_CC_regs)

.far       0    00803f78    00000218     
                  00803f78    00000140     rts6600e_elf.lib : defs.obj (.far) [fill = 0]
                  008040b8    0000006c     KeyStone_common.obj (.far) [fill = 0]
                  00804124    00000054     EMIF_main.obj (.far) [fill = 0]
                  00804178    00000010     KeyStone_common.obj (.far:Core_MPAX)
                  00804188    00000008     rts6600e_elf.lib : trgdrv.obj (.far) [fill = 0]

.cio       0    00804190    00000120     UNINITIALIZED
                  00804190    00000120     rts6600e_elf.lib : trgmsg.obj (.cio)

.neardata 
*          0    008042b0    0000009c     
                  008042b0    00000098     KeyStone_common.obj (.neardata)
                  00804348    00000004     KeyStone_EMIF16_Init.obj (.neardata)

.rodata    0    0080434c    00000000     UNINITIALIZED

.bss       0    0080434c    0000000c     UNINITIALIZED
                  0080434c    0000000c     EMIF_FLASH_mem_test.obj (.bss)

.cinit     0    00804358    00000290     
                  00804358    00000188     (.cinit..fardata.load) [load image, compression = rle]
                  008044e0    000000a1     (.cinit..neardata.load) [load image, compression = rle]
                  00804581    00000003     --HOLE-- [fill = 0]
                  00804584    0000001d     (.cinit..far.load) [load image, compression = rle]
                  008045a1    00000003     --HOLE-- [fill = 0]
                  008045a4    0000000c     (__TI_handler_table)
                  008045b0    00000008     (.cinit..bss.load) [load image, compression = zero_init]
                  008045b8    00000008     (.cinit..far:testBuf.load) [load image, compression = zero_init]
                  008045c0    00000028     (__TI_cinit_table)

.far:testBuf 
*          0    0c000000    00080000     UNINITIALIZED
                  0c000000    00080000     EMIF_main.obj (.far:testBuf)

.text      0    0c080000    00010300     
                  0c080000    00006740     KeyStone_common.obj (.text)
                  0c086740    00001ae0     flash_nand.obj (.text)
                  0c088220    00000800     EMIF_FLASH_mem_test.obj (.text)
                  0c088a20    000005c0     rts6600e_elf.lib : divd.obj (.text:__c6xabi_divd)
                  0c088fe0    000005c0                      : _printfi.obj (.text:_getarg_diouxp)
                  0c0895a0    00000520     KeyStone_common.obj (.text:Core_MPAX)
                  0c089ac0    000004e0     KeyStone_common.obj (.text:retain)
                  0c089fa0    00000460     rts6600e_elf.lib : _printfi.obj (.text:_printfi)
                  0c08a400    00000460                      : _printfi.obj (.text:_setfield)
                  0c08a860    000003a0     KeyStone_EMIF16_Init.obj (.text)
                  0c08ac00    000003a0     rts6600e_elf.lib : fputs.obj (.text:fputs)
                  0c08afa0    00000380     EMIF_main.obj (.text)
                  0c08b320    00000360     EMIF_NAND_FLASH_test.obj (.text)
                  0c08b680    00000320     rts6600e_elf.lib : _printfi.obj (.text:_pproc_fge)
                  0c08b9a0    000002e0                      : _printfi.obj (.text:_pproc_fwp)
                  0c08bc80    000002a0                      : _printfi.obj (.text:fcvt)
                  0c08bf20    00000280                      : divf.obj (.text:__c6xabi_divf)
                  0c08c1a0    00000280                      : _printfi.obj (.text:ecvt)
                  0c08c420    00000280                      : memory.obj (.text:free)
                  0c08c6a0    00000240                      : imath64.obj (.text:__c6xabi_divull)
                  0c08c8e0    00000240                      : _printfi.obj (.text:_pconv_e)
                  0c08cb20    00000240                      : _printfi.obj (.text:_pproc_diouxp)
                  0c08cd60    00000220                      : _printfi.obj (.text:_pproc_str)
                  0c08cf80    00000220                      : fputc.obj (.text:fputc)
                  0c08d1a0    00000200                      : _printfi.obj (.text:_pconv_g)
                  0c08d3a0    00000200                      : setvbuf.obj (.text:setvbuf)
                  0c08d5a0    000001c0                      : _printfi.obj (.text:_mcpy)
                  0c08d760    000001a0                      : trgdrv.obj (.text:HOSTrename)
                  0c08d900    000001a0                      : imath40.obj (.text:__c6xabi_divul)
                  0c08daa0    00000180                      : copy_decompress_rle.obj (.text:__TI_decompress_rle_core)
                  0c08dc20    00000180                      : memory.obj (.text:malloc)
                  0c08dda0    00000140                      : _printfi.obj (.text:_pproc_fflags)
                  0c08dee0    00000140                      : lowlev.obj (.text:getdevice)
                  0c08e020    00000120                      : fclose.obj (.text:_closefile)
                  0c08e140    00000120                      : _printfi.obj (.text:_ltostr)
                  0c08e260    00000120                      : fseek.obj (.text:fseek)
                  0c08e380    00000100                      : trgdrv.obj (.text:HOSTlseek)
                  0c08e480    00000100                      : autoinit.obj (.text:_auto_init_elf)
                  0c08e580    00000100                      : _io_perm.obj (.text:_wrt_ok)
                  0c08e680    00000100                      : cpy_tbl.obj (.text:copy_in)
                  0c08e780    000000e0                      : trgdrv.obj (.text:HOSTopen)
                  0c08e860    000000e0                      : divi.obj (.text:__divi)
                  0c08e940    000000e0                      : _printfi.obj (.text:_div)
                  0c08ea20    000000e0                      : atoi.obj (.text:atoi)
                  0c08eb00    000000e0                      : lowlev.obj (.text:close)
                  0c08ebe0    000000e0                      : copy_zero_init.obj (.text:decompress:ZI:__TI_zero_init)
                  0c08ecc0    000000e0                      : ltoa.obj (.text:ltoa)
                  0c08eda0    000000e0                      : memset.obj (.text:memset)
                  0c08ee80    000000e0                      : printf.obj (.text:printf)
                  0c08ef60    000000c0                      : trgdrv.obj (.text:HOSTread)
                  0c08f020    000000c0                      : trgdrv.obj (.text:HOSTunlink)
                  0c08f0e0    000000c0                      : trgdrv.obj (.text:HOSTwrite)
                  0c08f1a0    000000c0                      : divu.obj (.text:__divu)
                  0c08f260    000000c0                      : fflush.obj (.text:_doflush)
                  0c08f320    000000c0                      : exit.obj (.text:exit)
                  0c08f3e0    000000c0                      : tls.obj (.text:tls:init:__TI_tls_init)
                  0c08f4a0    000000a0                      : trgdrv.obj (.text:HOSTclose)
                  0c08f540    000000a0                      : fopen.obj (.text:_cleanup)
                  0c08f5e0    000000a0                      : _printfi.obj (.text:_ecpy)
                  0c08f680    000000a0                      : _printfi.obj (.text:_fcpy)
                  0c08f720    000000a0                      : memory.obj (.text:_minit)
                  0c08f7c0    000000a0                      : _printfi.obj (.text:_pconv_f)
                  0c08f860    000000a0                      : lowlev.obj (.text:finddevice)
                  0c08f900    000000a0                      : lowlev.obj (.text:lseek)
                  0c08f9a0    000000a0                      : memcpy64.obj (.text:memcpy)
                  0c08fa40    000000a0                      : memory.obj (.text:minsert)
                  0c08fae0    000000a0                      : memory.obj (.text:mremove)
                  0c08fb80    000000a0                      : lowlev.obj (.text:write)
                  0c08fc20    00000080                      : fixfu.obj (.text:__c6xabi_fixfu)
                  0c08fca0    00000080                      : llshift.obj (.text:__c6xabi_llshl)
                  0c08fd20    00000080                      : boot.obj (.text:_c_int00)
                  0c08fda0    00000080                      : trgmsg.obj (.text:readmsg)
                  0c08fe20    00000080                      : lowlev.obj (.text:unlink)
                  0c08fea0    00000060                      : cpp_init.obj (.text:__TI_cpp_init)
                  0c08ff00    00000060                      : frcmpyd_div.obj (.text:__c6xabi_frcmpyd_div)
                  0c08ff60    00000060                      : llshift.obj (.text:__c6xabi_llshru)
                  0c08ffc0    00000060                      : imath64.obj (.text:_subcull)
                  0c090020    00000060                      : memccpy.obj (.text:memccpy)
                  0c090080    00000060                      : trgmsg.obj (.text:writemsg)
                  0c0900e0    00000040                      : isinf.obj (.text:__c6xabi_isinf)
                  0c090120    00000040                      : _printfi.obj (.text:__c6xabi_isnan)
                  0c090160    00000040                      : strasg.obj (.text:__strasgi_64plus)
                  0c0901a0    00000040                      : args_main.obj (.text:_args_main)
                  0c0901e0    00000040                      : fputs.obj (.text:puts)
                  0c090220    00000020                      : negll.obj (.text:__c6xabi_negll)
                  0c090240    00000020                      : _lock.obj (.text:_nop)
                  0c090260    00000020                      : printf.obj (.text:_outc)
                  0c090280    00000020                      : printf.obj (.text:_outs)
                  0c0902a0    00000020                      : exit.obj (.text:abort)
                  0c0902c0    00000020                      : copy_decompress_none.obj (.text:decompress:none:__TI_decompress_none)
                  0c0902e0    00000020                      : copy_decompress_rle.obj (.text:decompress:rle24:__TI_decompress_rle24)


LINKER GENERATED COPY TABLES

__TI_cinit_table @ 008045c0 records: 5, size/record: 8, table size: 40
	.fardata: load addr=00804358, load size=00000188 bytes, run addr=00803b00, run size=00000474 bytes, compression=rle
	.neardata: load addr=008044e0, load size=000000a1 bytes, run addr=008042b0, run size=0000009c bytes, compression=rle
	.far: load addr=00804584, load size=0000001d bytes, run addr=00803f78, run size=00000218 bytes, compression=rle
	.bss: load addr=008045b0, load size=00000008 bytes, run addr=0080434c, run size=0000000c bytes, compression=zero_init
	.far:testBuf: load addr=008045b8, load size=00000008 bytes, run addr=0c000000, run size=00080000 bytes, compression=zero_init


LINKER GENERATED HANDLER TABLE

__TI_handler_table @ 008045a4 records: 3, size/record: 4, table size: 12
	index: 0, handler: __TI_decompress_rle24
	index: 1, handler: __TI_decompress_none
	index: 2, handler: __TI_zero_init


GLOBAL SYMBOLS: SORTED ALPHABETICALLY BY Name 

address    name
--------   ----
0c085584   Bus_error_handler
0c0902a0   C$$EXIT
0c0900d8   C$$IO$$
0c084a0c   EDMA_CC_error_handler
0c084c40   EDMA_TC_error_handler
0c086700   EDMA_TC_priority_cfg
0c0866c8   EDMA_channel_TC_cfg
0c0861d4   EDMA_copy
0c084de8   EDMA_error_handler
0c086328   EDMA_fill
0c086000   EDMA_init
0c085f80   EDMA_wait
00804348   EMIF16_Regs
0c08afa0   EMIF_init
0c085f6c   EXC_NMI
0c085e64   EXC_internal
0c085e50   EXC_swgen
0c089c2c   Exception_service_routine
0c088460   FLASH_MEM_AddrTest
0c08888c   FLASH_MEM_Bit_Walking
0c088220   FLASH_MEM_FillTest
0c088684   FLASH_MEM_Test
0080434c   FLASH_erase_blocks
00804354   FLASH_read_block
00804350   FLASH_write_block
0c083a60   Gauss_MPU4_constant
0c08f4a0   HOSTclose
0c08e380   HOSTlseek
0c08e780   HOSTopen
0c08ef60   HOSTread
0c08d760   HOSTrename
0c08f020   HOSTunlink
0c08f0e0   HOSTwrite
0c081900   IDMA_copy
0c085e14   IDMA_wait
0c084ed8   KeyStone_CIC_EXC_handler
0c084320   KeyStone_CIC_exception_events_mapping
0c085dc0   KeyStone_CorePac_AID_map
0c085d20   KeyStone_DDR_PLL_init
0c08a860   KeyStone_EMIF16_init
0c085694   KeyStone_EXC_external
0c084888   KeyStone_Exception_cfg
0c089688   KeyStone_MPAX_seg_setup
0c084144   KeyStone_MPU_MPPA_modify
0c083e8c   KeyStone_MPU_interrupts_enable
0c083ae0   KeyStone_MPU_range_setup
0c083b64   KeyStone_MPU_setup
0c083a10   KeyStone_MSMC_MP_interrupt_en
0c083920   KeyStone_MSMC_protection_exception_handler
0c08370c   KeyStone_PLL_init
0c0836cc   KeyStone_PrivID_Remap
0c0835ec   KeyStone_SES_MPAX_setup
0c08352c   KeyStone_SL2_EDC_enable
0c0831d0   KeyStone_SL2_EDC_handler
0c083184   KeyStone_SL2_EDC_interrupt_en
0c0830a0   KeyStone_SMS_MPAX_setup
0c089880   KeyStone_XMC_MPAX_setup
0c083000   KeyStone_disable_PSC_Power_Domain
0c082f6c   KeyStone_disable_PSC_module
0c082eb0   KeyStone_enable_PSC_module
0c082a68   KeyStone_main_PLL_init
0c082954   KeyStone_peripherals_MPU_excepiton_handler
0c082828   KeyStone_peripherals_MPU_fault_status
0c082798   KeyStone_print_device_info
0c082020   L1D_memory_protection_cfg
0c0826cc   L1P_EDC_setup
0c082524   L1P_ED_handler
0c081e60   L1P_memory_protection_cfg
0c082360   L1_MPPA_setup
0c0821c4   L1_cache_protection
00804334   LL2_EDC_DMA_err_str
00804338   LL2_EDC_L1D_err_str
0080433c   LL2_EDC_L1P_err_str
0c081bc0   LL2_EDC_handler
0c081ae4   LL2_EDC_scrub
0c081960   LL2_EDC_setup
00804330   LL2_EDC_victim_err_str
0c081740   LL2_MPPA_setup
0c081440   LL2_Memory_Protection_cfg
0c080a44   Memory_Address_Bus_Test
0c0811ac   Memory_Address_Test
0c080514   Memory_Data_Bus_Test
0c080f80   Memory_Fill_Test
0c0813c4   Memory_quick_test
0c08b5f8   NAND_FLASH_erase_blocks
0c08b514   NAND_FLASH_read_block
0c08b404   NAND_FLASH_test
0c08b320   NAND_FLASH_write_block
0c0880b0   NAND_eraseBlocks
0c08820c   NAND_globalErase
0c087fec   NAND_init
0c087b2c   NAND_isBadBlock
0c087ae0   NAND_protectBlocks
0c087350   NAND_readPage
0c087a24   NAND_unProtectBlocks
0c087928   NAND_verifyBlockErased
0c08788c   NAND_verifyPage
0c086d28   NAND_writePage
0c089ac0   Nested_Exception_service_routine
00803f60   Ns_str
00803f10   Peri_MPU_err_type_str
0c0801f0   Reset_Timer
0c0804f0   Service_Watchdog
0c080464   TN_MPU5_constant
0c0803ec   TSC_delay_ms
0c080370   TSC_delay_us
0c080330   TSC_init
0c080214   Timer64_Init
00804190   __CIOBUF_
008045c0   __TI_CINIT_Base
008045e8   __TI_CINIT_Limit
008045a4   __TI_Handler_Table_Base
008045b0   __TI_Handler_Table_Limit
UNDEFED    __TI_INITARRAY_Base
UNDEFED    __TI_INITARRAY_Limit
00803300   __TI_STACK_END
00001000   __TI_STACK_SIZE
008042b0   __TI_STATIC_BASE
00000800   __TI_SYSMEM_SIZE
UNDEFED    __TI_TLS_INIT_Base
UNDEFED    __TI_TLS_INIT_Limit
00000001   __TI_args_main
0c08fea0   __TI_cpp_init
0c0902c0   __TI_decompress_none
0c0902e0   __TI_decompress_rle24
00803f40   __TI_enable_exit_profile_output
ffffffff   __TI_pprof_out_hndl
ffffffff   __TI_prof_data_size
ffffffff   __TI_prof_data_start
0c08f3e0   __TI_tls_init
0c08ebe0   __TI_zero_init
ffffffff   __binit__
0c088a20   __c6xabi_divd
0c08bf20   __c6xabi_divf
0c08e860   __c6xabi_divi
0c08f1a0   __c6xabi_divu
0c08d900   __c6xabi_divul
0c08c6a0   __c6xabi_divull
0c08fc20   __c6xabi_fixfu
0c08ff00   __c6xabi_frcmpyd_div
0c0900e0   __c6xabi_isinf
0c08fca0   __c6xabi_llshl
0c08ff60   __c6xabi_llshru
0c090220   __c6xabi_negll
0c090160   __c6xabi_strasgi_64plus
ffffffff   __c_args__
0c08e860   __divi
0c08f1a0   __divu
0c090160   __strasgi_64plus
0c0901a0   _args_main
0c08e480   _auto_init_elf
0c08fd20   _c_int00
0c08f540   _cleanup
00803f38   _cleanup_ptr
0c08e020   _closefile
008020f8   _ctypes_
0c08f260   _doflush
00803f3c   _dtors_ptr
00803e84   _ft_end
00803b00   _ftable
00803f68   _lock
0c08f720   _minit
0c090240   _nop
0c089fa0   _printfi
00802300   _stack
0c08ffc0   _subcull
00803300   _sys_memory
00803f78   _tmpnams
00803f6c   _unlock
0c08e580   _wrt_ok
0c0902a0   abort
0c08ea20   atoi
ffffffff   binit
00803eb0   bus_err_stat_str
0c0801b8   calc_cycle_measure_overhead
0c08eb00   close
0c08e680   copy_in
00804328   cycle_measure_overhead
008040b8   exception_record
0c08f320   exit
0c08cf80   fputc
0c08ac00   fputs
0c08c420   free
0c08e260   fseek
00803ed0   gCIC_EXC_EN_MASK
00804344   gCIC_EXC_out_num
00804324   gDSP_Core_Speed_Hz
0080415c   gEmif16Cfg
00804140   gNandCeCfg
00803e38   gNandInfo
00804124   gNorCeCfg
008042b8   gpBootCfgRegs
008042b4   gpCGEM_regs
008042cc   gpCIC0_regs
008042d0   gpCIC1_regs
008042d4   gpCIC_regs
00804320   gpDDR_regs
008042d8   gpEDMA_CC2_regs
00803f70   gpEDMA_CC_regs
008042dc   gpEDMA_TC_2_0_regs
008042e0   gpEDMA_TC_2_1_regs
008042e4   gpEDMA_TC_2_2_regs
008042e8   gpEDMA_TC_2_3_regs
00803f28   gpEDMA_TC_regs
008042c8   gpGPIO_regs
00804310   gpMPU0_regs
00804314   gpMPU1_regs
00804318   gpMPU2_regs
0080431c   gpMPU3_regs
00803ef0   gpMPU_regs
008042c4   gpMSMC_regs
008042bc   gpPLLC_regs
008042c0   gpPSC_regs
008042ec   gpTimer0Regs
008042f0   gpTimer1Regs
008042f4   gpTimer2Regs
008042f8   gpTimer3Regs
008042fc   gpTimer4Regs
00804300   gpTimer5Regs
00804304   gpTimer6Regs
00804308   gpTimer7Regs
0080430c   gpTimer8Regs
00803e60   gpTimerRegs
008042b0   gpXMC_regs
00803df8   gstruMpuAddrRange
00804340   guwIntcCICExcEvtIdx
00803e88   internal_exception_str
0c08960c   lock_mem_prot_regs
0c08f900   lseek
0c08ecc0   ltoa
0c08b0e4   main
0c08dc20   malloc
00804178   mem_prot_key
0c090020   memccpy
0c08f9a0   memcpy
0c080000   memory_protection_exception_handler
0c08eda0   memset
0c08ee80   printf
0c0901e0   puts
0c08fda0   readmsg
0c08fe20   remove
0c08d3a0   setvbuf
0c000000   testBuf
00803f50   uiDataPatternTable
0080432c   uiLL2_scrub_addr
0c08fe20   unlink
0c0895a0   unlock_mem_prot_regs
0c08fb80   write
0c090080   writemsg


GLOBAL SYMBOLS: SORTED BY Symbol Address 

address    name
--------   ----
00000001   __TI_args_main
00000800   __TI_SYSMEM_SIZE
00001000   __TI_STACK_SIZE
008020f8   _ctypes_
00802300   _stack
00803300   __TI_STACK_END
00803300   _sys_memory
00803b00   _ftable
00803df8   gstruMpuAddrRange
00803e38   gNandInfo
00803e60   gpTimerRegs
00803e84   _ft_end
00803e88   internal_exception_str
00803eb0   bus_err_stat_str
00803ed0   gCIC_EXC_EN_MASK
00803ef0   gpMPU_regs
00803f10   Peri_MPU_err_type_str
00803f28   gpEDMA_TC_regs
00803f38   _cleanup_ptr
00803f3c   _dtors_ptr
00803f40   __TI_enable_exit_profile_output
00803f50   uiDataPatternTable
00803f60   Ns_str
00803f68   _lock
00803f6c   _unlock
00803f70   gpEDMA_CC_regs
00803f78   _tmpnams
008040b8   exception_record
00804124   gNorCeCfg
00804140   gNandCeCfg
0080415c   gEmif16Cfg
00804178   mem_prot_key
00804190   __CIOBUF_
008042b0   __TI_STATIC_BASE
008042b0   gpXMC_regs
008042b4   gpCGEM_regs
008042b8   gpBootCfgRegs
008042bc   gpPLLC_regs
008042c0   gpPSC_regs
008042c4   gpMSMC_regs
008042c8   gpGPIO_regs
008042cc   gpCIC0_regs
008042d0   gpCIC1_regs
008042d4   gpCIC_regs
008042d8   gpEDMA_CC2_regs
008042dc   gpEDMA_TC_2_0_regs
008042e0   gpEDMA_TC_2_1_regs
008042e4   gpEDMA_TC_2_2_regs
008042e8   gpEDMA_TC_2_3_regs
008042ec   gpTimer0Regs
008042f0   gpTimer1Regs
008042f4   gpTimer2Regs
008042f8   gpTimer3Regs
008042fc   gpTimer4Regs
00804300   gpTimer5Regs
00804304   gpTimer6Regs
00804308   gpTimer7Regs
0080430c   gpTimer8Regs
00804310   gpMPU0_regs
00804314   gpMPU1_regs
00804318   gpMPU2_regs
0080431c   gpMPU3_regs
00804320   gpDDR_regs
00804324   gDSP_Core_Speed_Hz
00804328   cycle_measure_overhead
0080432c   uiLL2_scrub_addr
00804330   LL2_EDC_victim_err_str
00804334   LL2_EDC_DMA_err_str
00804338   LL2_EDC_L1D_err_str
0080433c   LL2_EDC_L1P_err_str
00804340   guwIntcCICExcEvtIdx
00804344   gCIC_EXC_out_num
00804348   EMIF16_Regs
0080434c   FLASH_erase_blocks
00804350   FLASH_write_block
00804354   FLASH_read_block
008045a4   __TI_Handler_Table_Base
008045b0   __TI_Handler_Table_Limit
008045c0   __TI_CINIT_Base
008045e8   __TI_CINIT_Limit
0c000000   testBuf
0c080000   memory_protection_exception_handler
0c0801b8   calc_cycle_measure_overhead
0c0801f0   Reset_Timer
0c080214   Timer64_Init
0c080330   TSC_init
0c080370   TSC_delay_us
0c0803ec   TSC_delay_ms
0c080464   TN_MPU5_constant
0c0804f0   Service_Watchdog
0c080514   Memory_Data_Bus_Test
0c080a44   Memory_Address_Bus_Test
0c080f80   Memory_Fill_Test
0c0811ac   Memory_Address_Test
0c0813c4   Memory_quick_test
0c081440   LL2_Memory_Protection_cfg
0c081740   LL2_MPPA_setup
0c081900   IDMA_copy
0c081960   LL2_EDC_setup
0c081ae4   LL2_EDC_scrub
0c081bc0   LL2_EDC_handler
0c081e60   L1P_memory_protection_cfg
0c082020   L1D_memory_protection_cfg
0c0821c4   L1_cache_protection
0c082360   L1_MPPA_setup
0c082524   L1P_ED_handler
0c0826cc   L1P_EDC_setup
0c082798   KeyStone_print_device_info
0c082828   KeyStone_peripherals_MPU_fault_status
0c082954   KeyStone_peripherals_MPU_excepiton_handler
0c082a68   KeyStone_main_PLL_init
0c082eb0   KeyStone_enable_PSC_module
0c082f6c   KeyStone_disable_PSC_module
0c083000   KeyStone_disable_PSC_Power_Domain
0c0830a0   KeyStone_SMS_MPAX_setup
0c083184   KeyStone_SL2_EDC_interrupt_en
0c0831d0   KeyStone_SL2_EDC_handler
0c08352c   KeyStone_SL2_EDC_enable
0c0835ec   KeyStone_SES_MPAX_setup
0c0836cc   KeyStone_PrivID_Remap
0c08370c   KeyStone_PLL_init
0c083920   KeyStone_MSMC_protection_exception_handler
0c083a10   KeyStone_MSMC_MP_interrupt_en
0c083a60   Gauss_MPU4_constant
0c083ae0   KeyStone_MPU_range_setup
0c083b64   KeyStone_MPU_setup
0c083e8c   KeyStone_MPU_interrupts_enable
0c084144   KeyStone_MPU_MPPA_modify
0c084320   KeyStone_CIC_exception_events_mapping
0c084888   KeyStone_Exception_cfg
0c084a0c   EDMA_CC_error_handler
0c084c40   EDMA_TC_error_handler
0c084de8   EDMA_error_handler
0c084ed8   KeyStone_CIC_EXC_handler
0c085584   Bus_error_handler
0c085694   KeyStone_EXC_external
0c085d20   KeyStone_DDR_PLL_init
0c085dc0   KeyStone_CorePac_AID_map
0c085e14   IDMA_wait
0c085e50   EXC_swgen
0c085e64   EXC_internal
0c085f6c   EXC_NMI
0c085f80   EDMA_wait
0c086000   EDMA_init
0c0861d4   EDMA_copy
0c086328   EDMA_fill
0c0866c8   EDMA_channel_TC_cfg
0c086700   EDMA_TC_priority_cfg
0c086d28   NAND_writePage
0c087350   NAND_readPage
0c08788c   NAND_verifyPage
0c087928   NAND_verifyBlockErased
0c087a24   NAND_unProtectBlocks
0c087ae0   NAND_protectBlocks
0c087b2c   NAND_isBadBlock
0c087fec   NAND_init
0c0880b0   NAND_eraseBlocks
0c08820c   NAND_globalErase
0c088220   FLASH_MEM_FillTest
0c088460   FLASH_MEM_AddrTest
0c088684   FLASH_MEM_Test
0c08888c   FLASH_MEM_Bit_Walking
0c088a20   __c6xabi_divd
0c0895a0   unlock_mem_prot_regs
0c08960c   lock_mem_prot_regs
0c089688   KeyStone_MPAX_seg_setup
0c089880   KeyStone_XMC_MPAX_setup
0c089ac0   Nested_Exception_service_routine
0c089c2c   Exception_service_routine
0c089fa0   _printfi
0c08a860   KeyStone_EMIF16_init
0c08ac00   fputs
0c08afa0   EMIF_init
0c08b0e4   main
0c08b320   NAND_FLASH_write_block
0c08b404   NAND_FLASH_test
0c08b514   NAND_FLASH_read_block
0c08b5f8   NAND_FLASH_erase_blocks
0c08bf20   __c6xabi_divf
0c08c420   free
0c08c6a0   __c6xabi_divull
0c08cf80   fputc
0c08d3a0   setvbuf
0c08d760   HOSTrename
0c08d900   __c6xabi_divul
0c08dc20   malloc
0c08e020   _closefile
0c08e260   fseek
0c08e380   HOSTlseek
0c08e480   _auto_init_elf
0c08e580   _wrt_ok
0c08e680   copy_in
0c08e780   HOSTopen
0c08e860   __c6xabi_divi
0c08e860   __divi
0c08ea20   atoi
0c08eb00   close
0c08ebe0   __TI_zero_init
0c08ecc0   ltoa
0c08eda0   memset
0c08ee80   printf
0c08ef60   HOSTread
0c08f020   HOSTunlink
0c08f0e0   HOSTwrite
0c08f1a0   __c6xabi_divu
0c08f1a0   __divu
0c08f260   _doflush
0c08f320   exit
0c08f3e0   __TI_tls_init
0c08f4a0   HOSTclose
0c08f540   _cleanup
0c08f720   _minit
0c08f900   lseek
0c08f9a0   memcpy
0c08fb80   write
0c08fc20   __c6xabi_fixfu
0c08fca0   __c6xabi_llshl
0c08fd20   _c_int00
0c08fda0   readmsg
0c08fe20   remove
0c08fe20   unlink
0c08fea0   __TI_cpp_init
0c08ff00   __c6xabi_frcmpyd_div
0c08ff60   __c6xabi_llshru
0c08ffc0   _subcull
0c090020   memccpy
0c090080   writemsg
0c0900d8   C$$IO$$
0c0900e0   __c6xabi_isinf
0c090160   __c6xabi_strasgi_64plus
0c090160   __strasgi_64plus
0c0901a0   _args_main
0c0901e0   puts
0c090220   __c6xabi_negll
0c090240   _nop
0c0902a0   C$$EXIT
0c0902a0   abort
0c0902c0   __TI_decompress_none
0c0902e0   __TI_decompress_rle24
ffffffff   __TI_pprof_out_hndl
ffffffff   __TI_prof_data_size
ffffffff   __TI_prof_data_start
ffffffff   __binit__
ffffffff   __c_args__
ffffffff   binit
UNDEFED    __TI_INITARRAY_Base
UNDEFED    __TI_INITARRAY_Limit
UNDEFED    __TI_TLS_INIT_Base
UNDEFED    __TI_TLS_INIT_Limit

[249 symbols]
